:100C0000040C0E0C314020020B43C0430AF632C2E2
:100C1000F2C032000000B240805A2001F24085004C
:100C20005700F24080005600E2D32100E2D32200B8
:100C3000E2C32600E2C22A00E2C22E00B24010A5A2
:100C40002C01B24000A528013BC03A00B0127A0E38
:100C500082431202094336400A023742B012500F53
:100C6000C64C000016531783F92355420B027590AA
:100C700012007324759010006024B0124C0E55427F
:100C80000B0275901800302475901E00A4247590F6
:100C9000200016242BB21124759016002124759083
:100CA00014009F2475901A00172475901C00382496
:100CB000043CB012DA0EC23F2153B012E00EBE3F28
:100CC000B012DA0ED2420E025600D2420F02570084
:100CD000D24210021602B23FB012DA0E10420E02D9
:100CE00016420E021543073C3640FEFFB24006A5F1
:100CF000100235400C00B24000A52C0192421002B7
:100D00002801B643000092B32C01FD231583F32381
:100D10003690FEFFCE273740000236F000FE043C3E
:100D200016420E02174210023543759603201783B0
:100D3000FC23BF3F82460002C03F3640E0FF374001
:100D40002000B012500F7C9601242BD31783F92377
:100D50002BC2B0124C0E2BD2AC3F16420E021742E1
:100D600010022BB231243BD01000B012500F36903D
:100D70000010062C36900001092CC64C00001E3CC9
:100D8000B24000A52C01B24040A5280116B30320B3
:100D9000C24C1402133CC24C1502869AFDFF01247A
:100DA0002BD33690010204283BD23BB01000022422
:100DB0003BC032001A421402864AFFFF16531783C3
:100DC000D423B0124C0E753FB012500F1783FC2382
:100DD000B0124C0E723FB240F00F0E02B240100043
:100DE0001002B24080000A02D24210020C02D2422B
:100DF00010020D0282431202094336400A022742C2
:100E00007C46B012E40E1783FB2316420E021742F3
:100E10001002369000010A28B24614025C42140205
:100E2000B012E40E17835C421502013C7C46B012FE
:100E3000E40E1783EE23B2E312025C421202B012F8
:100E4000E40E5C421302B012E40EF83E18421202A5
:100E5000B012500FC24C1202B012500FC24C13020B
:100E600038E33BB20424869AFEFF01242BD3189268
:100E7000120222232BB320233041E2B22800FD27A7
:100E8000E2B22800FD23B24024026001E2B2280051
:100E9000FD27154270010511051105118245020259
:100EA000051182450402B2801E0004025742160258
:100EB00037800300051105111753FD23355040A558
:100EC00082452A013542B2402402600192927001AB
:100ED0000202FC2F1583F72309437C409000023C5B
:100EE0007C40A000C2430702C9EC120219E31BC3F5
:100EF000554207025545FA0E00550C2E2E2E2E2E69
:100F00002E2E2E1A3434924270017201B2500C000F
:100F10007201073C1BB30B208243620192B3620152
:100F2000FD27E2C321000A3C4C11F62B1BE3824350
:100F3000620192B36201FD27E2D3210092520202C4
:100F40007201D2530702F0900C00BDF2D123304160
:100F5000C24309021BC3554209025545600F0055A3
:100F60000C5656565656565656367600E2B228005D
:100F7000FD23924270017201925204027201824377
:100F8000620192B36201FD27E2B228001E282BD332
:100F90001C3C4C101A3C8243620192B36201FD2753
:100FA000E2B2280001281BE31BB301242BD3C9ECB8
:100FB000120219E30A3C8243620192B36201FD27E7
:100FC000E2B22800E62B4C101BE39252020272019F
:100FD000D2530902C03F8243620192B36201FD27EE
:100FE000E2B22800012C2BD33041FFFFFFFFFFFFAF
:100FF00011320040000000000000016001001212E8
:10100000FFFFFFFFFFFFFFFFFFFFFFFFFFFFFFFFF0
:10101000FFFFFFFFFFFFFFFFFFFFFFFFFFFFFFFFE0
:10102000FFFFFFFFFFFFFFFFFFFFFFFFFFFFFFFFD0
:10103000FFFFFFFFFFFFFFFFFFFFFFFFFFFFFFFFC0
:10104000FFFFFFFFFFFFFFFFFFFFFFFFFFFFFFFFB0
:10105000FFFFFFFFFFFFFFFFFFFFFFFFFFFFFFFFA0
:10106000FFFFFFFFFFFFFFFFFFFFFFFFFFFFFFFF90
:10107000FFFFFFFFFFFFFFFFFFFFFFFFFFFFFFFF80
:10108000FFFFFFFFFFFFFFFFFFFFFFFFFFFFFFFF70
:10109000FFFFFFFFFFFFFFFFFFFFFFFFFFFFFFFF60
:1010A000FFFFFFFFFFFFFFFFFFFFFFFFFFFFFFFF50
:1010B000FFFFFFFFFFFFFFFFFFFFFFFFFFFFFFFF40
:1010C000FFFFFFFFFFFFFFFFFFFFFFFFFFFFFFFF30
:1010D000FFFFFFFFFFFFFFFFFFFFFFFFFFFFFFFF20
:1010E000FFFFFFFFFFFFFFFFFFFFFFFFFFFFFFFF10
:1010F000FFFFFFFFFFFFFFFFFFFFFFFFFFFFFFFF00
:00000001FF
